:020000020000FC
:1000000006C04C7F406899C04D7F416896C000E0B3
:1000100002BB0FEF01BB0FEF08BB00E007BB662779
:10002000E0E0F2E17AD0402F0FEF8BD0EA9551F467
:10003000FA9541F4E0E0F2E167FF04C0142F106488
:1000400052D06F7742BB47FF02C0889A01C08898A0
:1000500006B342D016B3011749F701D0E7CF0E3FE0
:1000600081F20D3F79F10B3F79F2073FF9F00F3E36
:10007000F9F00F3D19F10F3B29F00F3759F00F3907
:1000800039F0089545FD02C017D057C013D055C0B0
:10009000112730C0042F0C70083011F418D04DC057
:1000A000003011F416D049C00FD047C0406145C0A0
:1000B0004F7E43C04F7D089540620895FDDF4E7F1F
:1000C00042683BC04C7739C048604B7F0895437FFE
:1000D00008954460477F089522E330E03A95F1F7B0
:1000E0002A95D9F708955FEF539521D0003069F034
:1000F0005F33D1F75FE30027E199FECF5EBB0DBB15
:10010000E19A5A955F3FB9F7EECFE199FECF5EBB1A
:100110001DBBE19A0BE415D0089550E45A9507D021
:10012000003009F008955030C9F700270895E1998B
:10013000FECF5EBBE09A0DB30895E0E0F2E16068A7
:1001400006E0969A12D0969810D00A95D1F742BB45
:1001500047FF02C0889A01C0889806B3BDDF16B376
:100160000117D9F70F3FC9F7089521E030E03A951C
:08017000F1F72A95D9F7089573
:00000001FF
:10018C005F7061E091DF5D2D5695569556955695AD
:10019C0062E08ADF5E2D5F7063E086DF09C05AE0A3
:1001AC0061E082DF5AE062E07FDF5AE063E07CDFEF
:1001BC001F910F914F9140935F00BF91AF914F9161
:0E01CC0018953F065B4F666D7D077F6F090833
:00000001FF
:1001DE0000E31ED00EE21CD00F910895A395B72F09
:1001EE00B770B295BA2BB93209F47064B83309F40A
:1001FE007064003321F070640BD0BCDF089576FF7D
:10020E0003C006D0B7DF0895AA3011F000E200C097
:10021E005D9BFECF0CB908950AE0FADF0DE0F8DF22
:10022E000895EF93FF93F2E0E0E40BD0FF91EF918E
:10023E0008956E666D7472303430393136410A0D60
:10024E000000C895002021F0002DE2DF3196F9CF95
:10025E0008950F930BE2DCDF0F9108950F931F9318
:10026E007F938F932FD0242F352F462F572F682F04
:10027E008F917F911F910F9108958F937F936F931D
:10028E005F934F932F913F914F915F916F918F910C
:10029E007F911F910F910895042F152F6FEF639586
:1002AE0000511742E0F75FE9505108511C4FE0F33F
:1002BE00539504561040E0F740EA4051065FE8F3CC
:1002CE00400F0895E9DF77278EEF4D5C43FF4350D3
:1002DE0047FF40535D5C53FF535057FF50536D5CC7
:1002EE0063FF635067FF6053220F331F441F551F78
:1002FE00661F771F881F4AF3111F18F77D5C73FF67
:10030E00735077FF70538D5F83FF8350DECF0F9353
:10031E000FB7319609F470680FBF0F9118950F93B0
:10032E000FB70F930BB10CB10F7D023599F0072F5C
:10033E0007700395053061F0787F702B706101E0D6
:10034E00902E602E702E802E0F910FBF0F9118954C
:10035E0001E0F2CF072F0770043049F700E00DBD22
:08036E000CBDEE27FF27F0CFC4
:00000001FF
